:020000040000FA
:020000000828CE
:020008000900ED
:10001000203084008001840A60300402031C0A2816
:100020002A16FF30C20041148316850185158312FC
:10003000850107309900C03083168100831231306A
:1000400090008E018F0100308B00003083168C00F1
:100050008312831631309B001C141A088312C500CA
:100060001B304502031C3528C50164000000D30B7A
:100070004F28851940280A30C207031847284F28FF
:1000800041184F280A30C202031C4B284F28411048
:10009000FF30C2004F284114C2018E214F288F0823
:1000A000031935288F0100304502031D60283F10D9
:1000B000BF10BF123F13A521012214222F2242227A
:1000C00001304502031D6D283F10BF10BF123F13C2
:1000D000A52101221422AF22422202304502031D33
:1000E0007A283F10BF10BF123F13A521012214220E
:1000F0002F22FB2203304502031D87283F10BF102B
:10010000BF123F13A52101221422AF22FB2204308B
:100110004502031D94283F10BF10BF163F17A521AD
:10012000012214222F22422205304502031DA1285C
:100130003F10BF10BF163F17A52101221422AF2286
:10014000422206304502031DAE283F10BF10BF16E5
:100150003F17A521012214222F22FB22073045023E
:10016000031DBB283F10BF10BF163F17A52101225A
:100170001422AF22FB2208304502031DC7283F107E
:10018000BF10BF163F17A5210122C7224222093006
:100190004502031DD3283F10BF10BF163F17A521EE
:1001A0000122C7229D220A304502031DDE283F148A
:1001B000BF10BF163F17A521C72242220B304502B0
:1001C000031DE9283F14BF10BF163F17A521C72202
:1001D0009D220C304502031DF5283F14BF10BF16A9
:1001E0003F17A52114222F2242220D304502031D64
:1001F00001293F14BF10BF163F17A5211422AF22BB
:1002000042220E304502031D0D293F14BF10BF16B8
:100210003F17A52114222F22FB220F304502031D78
:1002200019293F14BF10BF163F17A5211422AF2272
:10023000FB2210304502031D24293F14BF14BF16B2
:100240003F17A5211422422211304502031D2F29F8
:100250003F14BF14BF163F17A52114229D22123050
:100260004502031D3A293F14BF14BF163F17A521AD
:100270001422FB2213304502031D3F29DF211430D5
:100280004502031D4A293F14BF14BF163F17C02162
:100290002F22422215304502031D54293F14BF145A
:1002A000BF163F17C021B82216304502031D612931
:1002B0003F10BF10BF163F13A521012214222F2289
:1002C000422217304502031D6E293F10BF10BF1692
:1002D0003F13A52101221422AF22422218304502E9
:1002E000031D7B293F10BF10BF163F17A521012218
:1002F00014228B229D2219304502031D8429552288
:10030000672279228B229D221A304502031D8D29F6
:10031000552267227922AF229D223528C50A1B303B
:1003200045020318C5018B13450883161C159A0056
:1003300031309B0055309D00AA309D009C149C18C4
:100340009F291C1183128B170800B00A0A30300253
:10035000031C0800B11C8512B1180512FA30311CBB
:100360002D303002031C0800B10A3F1CB1100130CF
:10037000BF1EB100B11C8516B1180516B0010800EA
:10038000B00A0A303002031C08008512051205115C
:100390001E30B118643031198C303002031C080053
:1003A0000310B10DB1193114B1080319311431180A
:1003B0008516B118051631190515B0010800B00AE7
:1003C0000A303002031C0800851205120511851041
:1003D00005107D30311C53303002031C0800B10A77
:1003E0000330B105B1080319851603190516B118B4
:1003F0000515B11885143118FF29B1180514B0017D
:100400000800B20A0A303202031C08000512FF304D
:10041000331C37303202031C0800B30A01303F1F7F
:10042000B3000516B2010800B40A0A303402031CF6
:100430000800B51C0511B5188510F630351C323092
:100440003402031C0800B50ABF1CB51001303F1F61
:10045000B500B51C0515B5188514B4010800B60A19
:100460000A303602031C08008510F030381C1E309C
:100470003602031C0800B80A01303F1FB80085147B
:10048000B6010800B90A0A303902031C0800051039
:10049000F3303A1C28303902031C0800BA0A013034
:1004A0003F1FBA000514B9010800B00A1430311C0E
:1004B00046303002031C080085126730311C73304F
:1004C0003002031C0800B10A8516B0010800B20A08
:1004D0001430331C46303202031C0800051266300B
:1004E000331C72303202031C0800B30A0516B20135
:1004F0000800B40A1430351C46303402031C0800CE
:1005000005116230351C6C303402031C0800B50A3A
:100510000515B4010800B60A1430381C46303602FE
:10052000031C080085106730381C71303602031C2C
:100530000800B80A8514B6010800B90A14303A1C3C
:1005400046303902031C0800051064303A1C6E3036
:100550003902031C0800BA0A0514B901080036085C
:10056000B60B08000508023A8500C830B60008003E
:100570003608B60B0800B70A371C08000508023A0F
:1005800085000510851C0514A030B6000800A80FD2
:10059000D02A1E30A8000310AA0DAA1AAA15AA1262
:1005A0002808AB000130AA19AB0268302A050319EC
:1005B000DB2A851005152A132B080E020318E62ADC
:1005C00014302A050319E62A851405118F08031D26
:1005D000080064002B080E02031CE62A14302A05CA
:1005E0000319F42A8510051528302A050319FA2A5B
:1005F000851405110800A80F042B1E30A800031055
:10060000AA0DAA1AAA15AA122808AB000130AA1925
:10061000AB0268302A05031D05102A132B080E02B1
:100620000318162B14302A05031D05148F08031D0B
:10063000080064002B080E02031C162B14302A0538
:0E064000031D051028302A05031D05140800AF
:084000000000010001000300B3
:02400E00CC01E3
:00000001FF
